:104AAA00C2AF53FFBFE4F5F18EF38FF212000AAFE3
:064ABA00F443FF40D2AFFF
:014AC00022D3
:104A5D00C2AF53FFBF75F1A08EF38FF2AF058FF488
:0B4A6D0012000A43FF40D2AFAFF4225A
:104A2300C2AF53FFBF75F18012000A75F1308EF3E8
:0E4A33008FF2E4F5F412000A43FF40D2AF22E6
:01000A0022D3
:104B4400EEF0A3EFF0E4A3F0A3F022E0FEA3E0FF75
:024B5400C3227A
:1047070090242B124B4490242B124B4F90242EE0D5
:104717009F90242DE09E501A00000000000000002A
:10472700000090242EE004F070DC90242DE004F0CB
:0347370080D42209
:10479F00902427124B44902427124B4F90242AE049
:1047AF009F902429E09E50177FE87E0312470790C1
:1047BF00242AE004F070DF902429E004F080D7224F
:1047CF0090249A124B4490249A124B4F90249DE0C0
:1047DF009F90249CE09E50177F0A7E0012479F9067
:1047EF00249DE004F070DF90249CE004F080D72239
:104B5600759850438920438780758BFC758DFCD2F0
:024B66008E229D
:074BA100C298C299D2AC22B8
:084B99008F993099FDC29922A9
:102F3F00902439E0FEE42401FFEE3440FE22F090AD
:102F4F00244CE03400F0902442E0FF90243CE0FB5E
:102F5F00A3E0FAA3E0F9EF12153C902443E090248C
:102F6F003CFFE0FBA3E0FAA3E0F922902436E0FF58
:102F7F0090244CE0FCA3E0AA04F97B0022EFF0A31D
:102F8F00EBF0A3EAF0A3E9F0220B902452EBF0A3AD
:102F9F007424F0A37442F0A3E4F0A322FEE42411FE
:102FAF00FFEE3440FEA3E0FD22900001EF12154E1C
:102FBF00902444E090000212154E902445E09000BA
:102FCF000312154E902446E022902439E0FEE424AB
:102FDF0024FFEE3440FE22902439E0FEE42425FF46
:102FEF00EE3440FE22EFFD7C00E0FEE42DFFEC3ED0
:102FFF0022902439E0FEE42428FFEE3440FE229094
:10300F002439E0FEE42429FFEE3440FE22E4F0A34D
:10301F00F0A3F0A3F02225E024ABF582E43423F5EE
:10302F0083E022E0FF90244AE4F0A3EFF0E0FE22D9
:10303F00902447E07C002400FFEC3E229000030226
:10304F00150F902439E0FEE42404FFEE3440FE22F5
:10305F00E0FEE4240CFFEE3440FE0214F6FFEE34E3
:10306F0040FE90243A22E0FDA3E090244CCDF0A343
:10307F00EDF022E0FDA3E0902455CDF0A3EDF0227A
:10308F00FEF0FCA3EFF0FD22E0F9A3E0FAA3E0903D
:10309F002452C922E0FEE42400FFEE3440FE22E079
:1030AF00FFAA04A905902449E42290000102150FFC
:0630BF0090000202150F53
:103CDB00902439EFF090243BEAF0A3EBF090243AD8
:023CEB00EDF0FA
:103CED0064016018E0FF64026012EF6403600DEF81
:103CFD0064046008EF64056003023D95902439E08B
:103D0D00FF124A419024391230A390243DE0FD90DA
:103D1D00243AE04DFD124B0590243BE0FCA3E04C12
:103D2D00601C123051C006C007ECFDD007D0061242
:103D3D003DA02405FFEE3440FE90243B802B9024C3
:103D4D00A3E004F070069024A2E004F0123051C0FC
:103D5D0006C0079024A2E0FDD007D006123DA02496
:103D6D0005FFEE3440FE9024A2A3E0FD124B051298
:103D7D002F3F7D01124B05122F3F1249EFEF70F7C8
:103D8D0090243E7401F08005E490243EF090243E92
:023D9D00E0FF45
:0B3D9F0022124B05902439E0FEE422C4
:104A4100AB07EB122F437D10124B05EB122F4312D4
:0C4A510049EFEF70F6AF037DFF024B79D8
:0247FF00AA0707
:10480100124B1AEF6413701BEA122F437D02124BF5
:1048110005EA122F431249EFEF70F6902439740123
:0D482100F08005E4902439F0902439E0FF88
:01482E002267
:0538290090248CEFF07B
:10382E001214F6FFF470121230B9B4FF0C1230BF3E
:10383E00B4FF0612304BF4601CEF700F1230B970EB
:10384E000A1230BF700512304B600A902490E0705F
:10385E0002A3E07008E4902492F0023901902492C1
:10386E007401F090248C12305F12391A240D9000DE
:10387E0001123907240E900002123907240FFFEEB1
:10388E003440FE12304B12391A2410FFEE3440FE33
:10389E00C006C007902490E0FDD007D006124B055D
:1038AE0090248CE0902490122FAB124B051248BA44
:1038BE0090248C122F427D04124B0590248C122FD3
:1038CE00421249EFEF70F412392564156022123955
:1038DE00256417601B90248CE0FF124B90EF30E3B1
:1038EE00E690248CE0FF7D08124B79E4902492F050
:0838FE00124AD8902492E0FF69
:1039060022FFEE3440FE12150FFD124B0590248C5B
:10391600E0FEE422FD124B0590248CE0FEE42290AA
:10392600248CE0FEE42403FFEE3440FE1249EFEF60
:01393600226E
:104AEF00AB07EB122F437D08124B05EB122F43122E
:064AFF0049EFEF70F62202
:06338900902439122F8C84
:10338F0090243F12301CA3F0A3F0902439E0FE12DA
:10339F003025FCA3E0FD90243DE0FAA3E0FBD39D94
:1033AF00EA9C4011EE123025FDA3E0902443CDF0AE
:1033BF00A3EDF08008902443EAF0A3EBF0902439BA
:1033CF00E0FF124477902441EEF0A3EFF01234B8EF
:1033DF006417600EEF641C6009E4902443F0A3F0BF
:1033EF008015902443E0FCA3E0FDC3902442E09DB0
:1033FF00902441E09C40C6122FD81249EF90243FF1
:10340F00E4F0A3EFF0122FE61249EF902440122FB1
:10341F00F490243F12308F9024391230AE122F9037
:10342F0090244312307590243A122F71123937902D
:10343F002443E0FEA3E0FF902440E02FF090243FD0
:10344F00E03EF0122FD8C006C00790243FE0FDD019
:10345F0007D006124B05122FE690243FA3E0FD1272
:10346F004B05902439122F427D20124B05902439A1
:10347F00122F421249EFEF70F4902439E0FF124BF4
:10348F0090EF20E4111234B870EF902439E0FF125E
:10349F004A41E4FEFF22902439E0FF7D10124B7960
:0834AF00902443E0FEA3E0FFBE
:0B34B70022902439E0FF124B1AEF2294
:063DAA00902439122F8C59
:103DB00090243F12301CD390243EE0940090243D88
:103DC000E094005003023E641230001249EF902448
:103DD0003FE4F0A3EFF012300E1249EF90244012AE
:103DE0002FF490243F12308F902439E0FFAA04A9C9
:103DF000057B00C002C001A3123097122F909024BF
:103E00003D123082D001D002123A3690243DE0FEBD
:103E1000A3E0FF902440E02FF090243FE03EF0121A
:103E20003000C006C00790243FE0FDD007D0061246
:103E30004B0512300E90243FA3E0FD124B05902459
:103E400039122F427D40124B05902439122F421215
:103E500049EFEF70F490243DE0FFA3E0902441CFC0
:0C3E6000F0A3EFF0902441E0FEA3E0FF8F
:013E6C002233
:062D9200902434122F8C86
:102D9800E490243F12301D902434E0123025FEA325
:102DA800E0FF902438E0FCA3E0FDD39FEC9E902444
:102DB8003F4007EEF0A3EFF08005ECF0A3EDF090B4
:102DC800243A122F711214F6700F1230B9700A12C9
:102DD80030BF700512304B601490243DE07002A3A0
:102DE800E0600A90243FE07002A3E0700AE49024B7
:102DF8003FF0A3F0022F0090243412305F122F17F7
:102E0800240D12306C122F71900001122F09240E1C
:102E180012306C122F71900002122F09240F1230F9
:102E28006C122F7112304B122F172410FFEE344002
:102E3800FEC006C00790243DE0FDD007D006122F43
:102E48002EE090243D122FAB122F2E122FDB1249A9
:102E5800EF902441E4F0A3EFF0902434122FE9120C
:102E680049EFEFFD7C00902442122FF8FE90244198
:102E78001230909024341230AE122F9090243F12CA
:102E88003075902435122F7112393790243FE0FEA7
:102E9800A3E0FF902442E02FF0902441E03EF09020
:102EA8002434122FDBC006C007902441E0FDD00770
:102EB800D006124B05902434122FE9902441A3E048
:102EC800FD124B051248BA902434122F427D20126D
:102ED8004B05902434122F421249EFEF70F4122F51
:102EE8003520E40F122F3530E3F47D18122F22E439
:102EF800FEFF227D10122F2290243FE0FEA3E0FF68
:102F08002212150FFD124B05902434E0FEE422FD39
:102F1800124B05902434E0FEE422902434E0FF12A2
:102F28004B79124AD822124B05902434229024342B
:072F3800E0FF124B90EF22B5
:0630C500902436122F8C4E
:1030CB00E490244A12301DD390243BE094009024CA
:1030DB003AE0940050030232399024361230031236
:1030EB0049EF90244CE4F0A3EFF09024361230110A
:1030FB001249EFEFFD7C0090244D122FF890244CD9
:10310B00F0A3EFF09024361230A31249EFEF5407DF
:10311B0024FD605314607324026003023222122FC9
:10312B007AC003122F987408F0D00312324224088D
:10313B00122F4D122FB890243F122F70E48FF012E4
:10314B0015FF90243F122F7112159CFE12303F8FEA
:10315B00F01215FF902448123032902449E02400DD
:10316B00FFEC3EA30231C8122F7AC003122F9874C2
:10317B0006F0D0031232422406122F4D122FB81232
:10318B00303312303F90244A8033122F7AC003120F
:10319B002F987402F0D003123A3690244DE024029B
:1031AB00F090244CE03400F0902442123032902402
:1031BB0043123042CF24FECF34FF90244AF0A3EFCA
:1031CB00F0122F7AC002C001902437123097122FC1
:1031DB009090244A123082D001D002123A369024B9
:1031EB004AE0FEA3E0FF90244DE02FF090244CE04A
:1031FB003EF0902436123003C006C00790244CE0FA
:10320B00FDD007D006124B059024361230119024B6
:10321B004CA3E0FD124B05902436122F427D401239
:10322B004B05902436122F421249EFEF70F4902485
:06323B004AE0FEA3E0FFE3
:0932410022123A3690244DE022DD
:0B45A1004823BB0000000000000000E9
:10324A00902433E025E0FF902432E033FE74AB2F64
:10325A00F58274233EF58322902433E025E0FF9023
:10326A002432E033FE749B2FF58274233EF58322C9
:10327A00AC02AD03C39DFFEE9CF0A3EFF0A3E0FE0A
:10328A00A3E0FFE422F0A3E4F0748B2FF582742309
:10329A003EF58322F0A3E4F0747B2FF58274233E7B
:1032AA00F58322FFEE3440FEE0FBA3E0FAA3E0F947
:1032BA008D828C8312150FFD124B05902432E0FC8F
:1032CA00A3E0FD222FFFE43EFEED34FEFDEC338F3A
:1032DA000F8E0E8D0DF50C2225E024C7F582E434FD
:1032EA0023F583E0FEA3E0222FFFE43EFEE434FE52
:1032FA00FDE433FC227A00AB07E0FEE422E0F5109D
:10330A00A3E0F51122EFFD7C00EBFEE42DFBEC3E81
:10331A00FA4B228F0F8E0EF50DF50C22F583E05A2B
:10332A00FEA3E05FFBAA06E922FEE42DFFEC3EF0D5
:10333A00A3EFF022F583E0FCA3E0C39FEC9E22C238
:10334A00AF7593FE8F828E8322EFF0E4A3F0A3F091
:10335A00FBFA22902439E0FEE422A3E0FAA3E0FF7C
:10336A002225E024D7F582E434232225E024ABF594
:0F337A0082E434232225E0249BF582E4342322CD
:104AC100124BAEC2AF124B5675EBFF75ECFF75ED95
:074AD100FF75EEFFD2AF22DA
:044BAE0075FF40222D
:104B680075FE0843FE207F647E0012479F53FEDFD8
:014B7800221A
:104B0500A2AFE433FC123349EDF0E4F593AF04EFC3
:044B150024FF92AF38
:014B19002279
:0D49E200902445E0FEE42420FFEE3440FE6A
:1049EF00A2AFE433F9123349E0FFE4F593AD01EDE3
:0449FF0024FF92AF50
:014A03002290
:094B9000EFFEE424021249EA22BE
:0D4B7900EFFEE42402FFEE3440FE024B0587
:0B261F0090242CEBF0A3EAF0A3E9F0FC
:10262A00E4902434F0A3F0A3F0A3F09023D77480AD
:10263A00F0A3E4F09023C774C0F0A3E4F09024322E
:10264A00F0A3F01232C5FEE4241F90242C1232ADFE
:10265A00FEE4241E90242F1232AD25E0FFEC123244
:10266A0055E4F0A3F012326FE4F0A3F0C3902434DF
:10267A00E0648094C0506790242CE0FBA3E0FAA3A6
:10268A00E0F98D828C8312150F24FE601D24FE60F2
:10269A002624FC602E24F86036240F704112324A38
:1026AA00740412328F74030226E312324A74081237
:1026BA00328F74070226E312324A741012328F7470
:1026CA000F801612324A742012328F741F800A1237
:1026DA00324A744012328F743FF0A374FFF0C390F1
:1026EA002436E0648094C0507290242FE0FBA3E06B
:1026FA00FAA3E0F9A3E0FEA3E0FFF5828E831215A8
:10270A000F24FE602224FE602B24FC603324F86030
:10271A003B240F7046EF25E0FFEE12326D7404126F
:10272A00329E7403022760123262740812329E7457
:10273A0007022760123262741012329E740F8016DA
:10274A00123262742012329E741F800A123262742C
:10275A004012329E743FF0A374FFF01232C525E096
:10276A00FFEC123255E0FAA3E0FB902435E02BF09F
:10277A00902434E03AF012326FE0FEA3E0FF902496
:10278A0037E02FF0902436E03EF0ED4C607B902449
:10279A0032A3E025E0FFEC33FE74A92FF5827423FF
:1027AA003EF583E0FAA3E0FB74D52FF58274233E4D
:1027BA001232EB2BFBEE3AFAED25E0FFEC33FE7416
:1027CA00D72FF58274233EF583EAF0A3EBF07499D0
:1027DA002FF58274233EF583E0FCA3E0FD74C52F38
:1027EA00F58274233E1232EB2DFDEE3CFC9024332D
:1027FA00E025E0FF902432E033FE74C72FF582749F
:10280A00233EF583ECF0A3EDF0902433E004F0705E
:10281A0006902432E004F0C3902433E09408902414
:0B282A0032E064809480500302264DD1
:012835002280
:024B1A00AC07E6
:104B1C007BFFECFEE424031249EAEF6B6004AB0765
:024B2C0080F017
:014B2E002264
:0344770090244549
:10447A001233531249E29024451232FF2421124981
:10448A00EA12330F60221249E2902446E4F0A3EFC5
:10449A00F0902445E0FEE424211249EAEFFD90243D
:1044AA0047E0902446123333902446E0FEA3E0FF0F
:0744BA006B7002EE6A70BC9A
:0144C10022D8
:03442500902439A7
:1044280012335312335D24261249EA90243912328A
:10443800FF24271249EA12330F602412335D242621
:104448001249EA90243AE4F0A3EFF012335D2427EE
:104458001249EAEFFD90243BE090243A123333905E
:0E446800243AE0FEA3E0FF6B7002EE6A70B52E
:014476002223
:05393700902445EFF0B3
:10393C00AF01902450EAF0A3EFF0902449123364C5
:10394C00902445E0F925E0248BF582E434231233EE
:10395C002612336B1232EB2BFFEE3A902452F0A36B
:10396C00EFF090244DE02BFF90244CE03AFEE9124E
:10397C00337512333E4003023A0E902445E0123365
:10398C00751232EB90244E12327AFCFDC004C00545
:10399C00C006C0071232871232CE90244E12330763
:1039AC00D007D006D005D00412430790244EE0FE79
:1039BC00A3E0FF902451E02FF0902450E03EF0C3A0
:1039CC0090244DE09FFF90244CE09E90244EF0A359
:1039DC00EFF0902445E012336BF583E0FFA3E09009
:1039EC002452CFF0A3EFF0902450123288FCFDC08B
:1039FC0004C005C006C0071232871232CE90244E86
:103A0C008019902450123288FCFDC004C005C006F9
:103A1C00C0071232871232CE90244C123307D007D3
:093A2C00D006D005D004124307B6
:013A3500226E
:0E3A360090244EEFF0A3EBF0A3EAF0A3E9F02A
:103A4400A312336490245BEAF0A3EFF090244F12A6
:103A5400336490244EE0F925E0247BF582E434239A
:103A64001233261232E22BFFEE3A902459F0A3EFE0
:103A7400F0902456E02BFF902455E03AFEE91233EF
:103A84007F12333E507490244EE012337F1232EB97
:103A940090245712327A1232F2C006C007123287CB
:103AA40012331D902457123307D007D00612430750
:103AB400902457E0FEA3E0FF90245CE02FF09024D4
:103AC4005BE03EF0C3902456E09FFF902455E09EB7
:103AD400902457F0A3EFF090244EE01232E2FF90CE
:103AE4002459EEF0A3EFF0E41232F2C006C007123C
:103AF400328712331D90245780169024591232882D
:103B04001232F2C006C00712328712331D902455B8
:0A3B1400123307D007D00612430752
:013B1E002284
:1048E4001214F69023C3F090000112150F9023C404
:1048F400F090000212150F9023C5F09000031215DA
:064904000F9023C6F02213
:1048BA009023C3E0FD7F057E00124B059023C4E0E0
:1048CA00FD7F06124B059023C5E0FD7F07124B05BD
:0A48DA009023C6E0FD7F08024B05A5
:104AD800E4FD7F05FE124B057F06124B057F07128A
:074AE8004B057F08024B059E
:104930009023C3E012153C9023C4E09000011215AF
:104940004E9023C5E090000212154E9023C6E090D1
:05495000000302154EFA
:104307008F0B8E0A8D098C08A2AFE433F5148593C1
:104317001578101216FDA907AF0FAE0EAD0DAC0C38
:1043270078101216FDAB07C2AFE5111511AE10706C
:104337000215104E6022899378081217408F828EDB
:1043470083E0751200F5138B93AA13780C121740AC
:104357008F828E83EAF080D1E51424FF92AF851512
:0243670093229F
:1034C2000D414343455320492F4F2050726F64757D
:1034D2006374732C20496E632E0D0A4D6F64656C04
:1034E200204554482D44494F2D3438204669726D89
:1034F20077617265205265766973696F6E20256205
:10350200782E256278206275696C643A25732040B2
:10351200202573200D0A0030312F31392F3233002C
:1035220030393A35303A3535004D41432041444433
:103532005245535320495020202020203A20252E46
:103542003262782E252E3262782E252E3262782E25
:10355200252E3262782E252E3262782E252E326268
:10356200780D0A005355424E4554204D41534B208D
:10357200202020202020203A20252E3362752E255F
:103582002E3362752E252E3362752E252E336275EB
:103592000D0A0047617465776179204950204144E2
:1035A2004452455353203A20252E3362752E252E40
:1035B2003362752E252E3362752E252E3362750DDC
:1035C2000A004950204144445245535320202020B0
:1035D20020202020203A20252E3362752E252E33DE
:1035E20062752E252E3362752E252E3362750D0AD5
:0135F20000D8
:1045AC004101140048010B080201010101010148FD
:0F45BC000103080201010101010142000000009A
:034BB200C2B72265
:034BB500D2B72252
:101F2400124BB212473A90242F7401F0A37401F0BB
:101F3400A37403F07B017A01790B12261F90243AD3
:101F44007401F0A37450F0A374FFF0A37435F0A3EC
:101F54007419F0A374FFF0A37435F0A37422F07B1A
:101F6400FF7A3479C212193E1221A21221A212411F
:101F74004E12218A7F327E0012479F124BB27F326B
:101F84007E0012479F12218A7F287E0012479F12EB
:101F94004BB27F097E001249EFC0077F0A7E001210
:101FA40049EFC0077F0B7E001249EFAC077F0C7E20
:101FB400001249EFAB077F0D7E001249EFAA077F9D
:101FC4000E7E001249EF90243FEFF090243EEAF099
:101FD40090243DEBF090243CECF090243BD0E0F0D6
:101FE40090243AD0E0F07BFF7A35792B12193E7FAA
:101FF400057E001249EF7F067E001249EF7F077EBF
:10200400001249EF7F087E001249EF7F017E001223
:1020140049EF7F027E001249EF7F037E001249EFF1
:102024007F047E001249EF7F0F7E001249EFAC0758
:102034007F107E001249EFAB077F117E001249EF3B
:10204400AA077F127E001249EF90243DEFF09024FE
:102054003CEAF090243BEBF090243AECF07BFF7ADE
:102064003579C412193E9001157401F07A007B028F
:102074007DE17CCAE4FF120EB87F011221767F0253
:102084001208007F031221767F041221B77F051204
:1020940021B77F061208007E017F161237141246FC
:1020A400229024A5E0602614F07F017E0012479F51
:1020B4009024A5E070177B017A2479131249BF7A22
:1020C40024791712499C7A24791B124979A2893000
:1020D4008B01B35032308B0E902117E0700804F05E
:1020E400124558122127208B05E4902117F03089DE
:1020F4000E902116E0700804F012482F12212720B8
:102104008905E4902116F0900102E0640160030265
:10211400207090213FE0640160030220701221C30B
:102124000220707B017A2479131249BF7F0F7E004D
:102134001249EFAC077F107E001249EFAB077F1105
:102144007E001249EFAA077F127E001249EF902405
:102154003DEFF090243CEAF090243BEBF090243ADD
:10216400ECF07BFF7A3579C412193E9001157401A5
:10217400F0227A017B167DE07CCA1208007A017B8A
:10218400167DE07CCA22124BB57F327E0012479F37
:10219400124BB27F327E0012479F124BB5227F64EE
:1021A4007E0012479F124BB57F647E0012479F1238
:0F21B4004BB2221208007A017B167DE07CCA2212
:10473A00E4902117F0902116F0124BAEC2AF75FF2C
:10474A0028F59DF59E758E02759203759C3F124A57
:10475A0092124B5675EBFF75ECFF75EDFF75EEFF88
:03476A00D2AF22A9
:03002300024BA8E5
:064BA800309802C29832B1
:10462200900000E07002A3E0601A90000074FFF5B1
:10463200F0121570FEC3E5F09440EE648094805051
:104642001A024BB2900115E06011900000E4F0A351
:0B4652007480F0124BB5E4900115F0ED
:01465D00223A
:10465E000D0A3E20444843502053756363657373BF
:10466E002E0D0A000A0D3E20444843502046616933
:10467E006C2E00202D207374617274696E67204455
:0A468E004843500D0A000000000030
:1044C2009001157401F09024077482F0A3F0A3F018
:1044D200A3F0E4A3F02290240B7401F0A37450F033
:1044E2007B017A2479072274C0F074A8A3F0A37424
:1044F20001F02290000112150FFD22900002121508
:0B4502000FFD2290000312150FFD2298
:0B45E500902439EBF0A3EAF0A3E9F00A
:1045F000E4A3F090243CE0FD2409FFE433FE902482
:1046000039E0FBA3E0FAA3E0F98D8275830012156F
:104610000FFD124B0590243CE004F0E0C3940640EB
:01462000D2C7
:014621002276
:104979001214F6FD7F017E00124B051244F57F02E9
:10498900124B051244FD7F03124B051245057F04A6
:03499900024B05C9
:10499C001214F6FD7F057E00124B051244F57F06BE
:1049AC00124B051244FD7F07124B051245057F087B
:0349BC00024B05A6
:1049BF001214F6FD7F0F7E00124B051244F57F1087
:1049CF00124B051244FD7F11124B051245057F1244
:0349DF00024B0583
:103B1F0078287C247D017BFF7A4679947E007F0490
:103B2F001214D07D80E4FFFE124B0590240DE0FDB2
:103B3F007F09124B0590240EE0FD7F0A124B059072
:103B4F00240FE0FD7F0B124B05E4FD7F0C124B059C
:103B5F007F0D124B057F0E124B057F01123BE57F48
:103B6F0002124B057F03123BF37F04124B057F05B7
:103B7F00123BE57F06124B057F07123BF37F0812BE
:103B8F004B05902428E0FD7F0F124B05902429E070
:103B9F00FD7F10124B0590242AE0FD7F11124B057B
:103BAF0090242BE0FD7F12124B057D177F17124BD0
:103BBF00057D707F18124B057D037F19124B059001
:103BCF00242F7401F0A37401F0A37403F07B017A26
:063BDF0001790B02261F14
:103BE500902428E0FD124B05902429E0FD22902425
:0C3BF5002AE0FD124B0590242BE0FD227D
:10482F001244C2A3F09024131244E9A374AEF0A370
:10483F0074FF1244CFA31244E9745E1244EEE49065
:0F484F0024261244E1124A049021167401F0222B
:104558001244C2A3F0A3F0A37408F0A374DCF0A380
:104568007411F0A37499F0A37477F0A3740AF0A3FC
:104578007401F0A3F0A374FBF0A374FF1244CFA35B
:10458800740AF0A374011244CF9024261244E11255
:094598004A049021177401F0227D
:1046D0001244E2124B8690240BE0B40106A3E0647E
:1046E0005060061244D8124A047B017A24791312CE
:1046F00049BF7A24791B1249797A24791712499C87
:074700007A24790D0245E562
:1043CA00124369EF601490213F7401F07BFF7A4633
:1043DA00795EE490243AF002193EE490213FF07BA2
:1043EA00FF7A46797290243AF012193EE4FF741B60
:1043FA002FF582E43424F583E4F074172FF582E470
:10440A003424F583E4F074132FF582E43424F5831D
:0A441A00E4F00FEFB404D712000025
:014424002275
:10414E001246D030892B308B287BFF7A467981122C
:10415E00193E9001027401F0123B1F1243CA9001E6
:10416E0002E06401705890213FE06401705002211A
:01417E00C37D
:10417F00902407E0FF902427F0BF8203308B0512B5
:10418F004558801B30890512482F801390240BE06F
:10419F00B40106A3E0645060061244D8124A047BAF
:1041AF00017A2479131249BF7A24791B1249797A3B
:0D41BF0024791712499C7A24790D1245E5E8
:0141CC0022D0
:104B2F00AE028EFB8FFAE4FBFDFC22EBF0A3EAF062
:054B3F00A3E9F0E422EF
:10488D00E490243CF0A2AF33F0C2AF53FFBF8FF1E1
:10489D00AE04AF058EF38FF2AF038FF41207FD4315
:0C48AD00FF4090243CE024FF92AFAFF4E9
:0148B90022DC
:104A0400902439124B3AFBFDFC7FD012488D902440
:0F4A140039A3E0FAA3E0FF124B2F7FD102488DA8
:0A4B8600AF01124B2F7FD202488DC1
:10495500AC02AD018CFB8DFA902498E0FCA3E02914
:10496500F9EA3CAD01F5FD8DFCAD07AC06E4FB7F36
:04497500A102488DC6
:0941CD00902483EEF0A3EFF0A3AF
:1041D600124B3A90248AF0A3F0902488E0FEA3E0E4
:1041E600FFA3E0FCA3E0FDC39FEE6480F8EC6480CF
:1041F600985041902484E02DFF902483E03CCF2406
:10420600FFCF34FF8F82F583740193FF902485E0FE
:10421600FBA3E0FAA3E0F990248AA3E0F5828C835D
:10422600EF12154E90248BE004F070AD90248AE0D6
:0442360004F080A56B
:01423A002261
:10700000C2AF75FF407F717E001271D17F617E003B
:107010001271D1E4900000F0A3F0FFFE1271B77F6F
:10702000007E681271B753FFBF75F18012000A75B8
:10703000F130900000E0FEA3E0FF8EF38FF2E4F564
:10704000F412000A43FF401271AF53FFBF75F1A065
:10705000900000E0FEA3E0FF8EF38FF2E42FF582B4
:1070600074803EF583E0F5F412000A43FF4090007F
:1070700001E004F07006900000E004F0D3900001FD
:10708000E09400900000E0946840097F317E001297
:1070900071D1800C900000E05403FEA3E04E70AA72
:1070A000A2A2B392A2A2A3B392A3C3900000E094C1
:1070B0006850030270267F427E001271D1E4900076
:1070C00000F0A3F01271AFC20020003853FFBFE4FC
:1070D000F5F1900000E0FEA3E0FF8EF38FF21200C6
:1070E0000AAFF443FF40900000E0FCA3E0FDE42D74
:1070F000F58274803CF583E06F6009D2007F437EA7
:10710000001271D1900001E004F07006900000E0E0
:1071100004F0D3900001E09400900000E0946840F7
:10712000097F327E001271D1800C900000E0540380
:10713000FEA3E04E7093C200A2A2B392A2A2A4B397
:1071400092A4C3900000E0946850030270C4C2A2ED
:10715000D2A3D2A47F7A7E001271D1020000AD07C3
:10716000EDC4540FFFC3940A400BEF75F00A84E599
:10717000F02441800CEDC4540F75F00A84E5F0242E
:1071800030FFE433FE1271D1ED540FFFC3940A4077
:107190000BEF75F00A84E5F02441800BED540F7578
:1071A000F00A84E5F02430FFE433FE1271D122901E
:1071B0000000E0FEA3E0FFAB07AA06EAFF12715E43
:1071C000AF0312715E7F0D7E001271D17F0A0271D2
:0971D000D18F993099FDC299227A
:102BDC002406F582E43EF583E0FD7F007E801246FC
:102BEC00C190242AE0FEA3E02407F582E43EF5839D
:102BFC00E0FD7F017E801246C190242AE0FEA3E016
:102C0C002408F582E43EF583E0FD7F027E801246C7
:102C1C00C190242AE0FEA3E02409F582E43EF5836A
:102C2C00E0FD7F037E801246C190242AE0FEA3E0E3
:102C3C00240AF582E43EF583E0FD7F047E80124693
:102C4C00C190242AE0FEA3E0240BF582E43EF58338
:102C5C00E0FD7F057E801246C1902430E0FBA3E0AE
:102C6C00FAA3E0F9740512153C902430E0FBA3E0C4
:102C7C00FAA3E022740490000512154E902427E06C
:102C8C00FF90242AE0FCA3E0AA04F97B0190243DE8
:102C9C00E4F0A32290242EE0FEA3E0FF240CFDE43C
:102CAC003EFC90242AE0FAA3E0FB2DF582EA3CF5E9
:102CBC0083E0F9902437F0EF2406FFE43EFEEB2F7F
:102CCC00F582EA3EF583E0902438F0FEE95E90242C
:102CDC0037F0EEF4A3F0222407F9E43AFA0D024897
:102CEC007DF990000512150F902413F09000061238
:102CFC00150F902414F090000712150F902415F066
:102D0C0090000802150F9001157401F022E0FF905D
:102D1C00242AE0FCA3E0AA04F97B012290000574AC
:102D2C000612154EE92406F9E43AFA7D007C80027D
:102D3C00487DF090000602150FC390242FE09406F6
:102D4C0090242EE0940022F9900001021710902498
:102D5C002AE0FEA3E022902433E02400FFE4348038
:102D6C00FE22E490242EF0A3F022F9900005021527
:102D7C000FF090000702150F90242FE004F0229022
:062D8C00242EE004F022F9
:10469800F990242EE0FEA3E0FF240CF582E43EF519
:1046A8008312150FFD902438E05DFD902437E04D0E
:0946B800FDF0E42FFFEE3480FE5A
:0446C1008F828E83D3
:0A46C500AF05759301EFF0E4F593E3
:0146CF0022C8
:10485E00F990242EE0FEA3E0FF240CFDE43EFCE9DB
:0F486E002DF9EA3CFAE42FFFEE3480FEAD07FC93
:04487D008D828C8319
:0C488100759301E0FFE4F593EF02153C95
:10080000902427EFF0A3ECF0A3EDF0A3EAF0A3EB24
:01081000F0F7
:10081100F99024307401F0A3EAF0A3E9F0E4902404
:1008210036F0902427E0FF124B1AEF7003020E5DA1
:1008310024ED7003020E7B24F77003020E5524058C
:100841006003020E83902427E0FF124B90EF30E00B
:010851004C5A
:10085200E4902437F0902437E0FFC394065033909D
:100862002427E0FEEF6E6022902437E0FF124B1A3D
:10087200BF1717E490242CF0A3F0902437122D19FF
:10088200E490243DF0A3F0123389902437E004F081
:0C08920080C3902427E0FF7D01124B7909
:10089E00902427E0FF12442590242CEEF0A3EFF0D5
:1008AE00D39400EE94005003020E83902427122D51
:1008BE0019A3E0FDA3E090243DCDF0A3EDF0123D91
:1008CE00AA90242CEEF0A3EFF0122C75122D5312D9
:1008DE0017C10BBD436847570B644368494F0B96CE
:1008EE00436849500CDE43684D430C3B43684E5001
:1008FE000C3B43684E570BFC4368534D0A65444905
:10090E004F2109FC5241444909505241445309AB0D
:10091E005241574C0E34525044490D3A5253746161
:10092E000E13554461740E175546696E0A80574171
:10093E00444F0AA15750444F0ADE5752504400000C
:10094E000E34122D12122C75F9740D122C72F990A0
:10095E00000112179D525F4F4B122D28122C75124B
:10096E002CE3122C752408122CE5122C7524091276
:10097E002CE5122C75240A122CE5122C75240B1260
:10098E002CE5122C75F990000C740112154EE5B081
:10099E00543F90000D122C85740E020E31902436A9
:1009AE007401F0122D5A2406F582E43EF583E0FF21
:1009BE00131313541FFE902433F0EF5407A3F07B50
:1009CE00017A247935EE2400FFE4124877122D6265
:1009DE00902435E0FD902434E0FC7401A8040880D6
:1009EE0002C333D8FC6DFD902435F01246C1122D92
:1009FE0012122C75F9740B122C72F9900001121749
:100A0E009D525F4F4B122D28122C75122CE3122C77
:100A1E00752408122CE5122C752409122CE5122CC3
:100A2E0075240A122CE5122C75240B122CE5902439
:100A3E0036E0601B122D62A3E0FD7401A80508804C
:100A4E0002C333D8FCFD902435E06DFD1246C11271
:100A5E002C88740C020E31122D12122C65F9900096
:100A6E000112179D5F4572727432122C8274060247
:100A7E000E31122D12122D5A122BDCF9900001128A
:100A8E00179D575F4F4B9000057406122C85740608
:090A9E00020E31122D12122D6E10
:0F0AA700122CA0122C7512485E122C7512469854
:100AB600122D847003122D8B122D4540E4122C65E5
:100AC600F990000112179D575F4F4B900005740671
:0E0AD600122C857406020E31122D12122D6E96
:100AE400122CA0122C7512485E122C751246981204
:100AF4002C75F990242EE0FEA3E0FF240612486929
:100B0400122D847003122D8B122D4540D3122C7597
:100B1400122D537B4F7A4479507857C31216EC90B8
:100B24002430701B122C68F990000112179D575F36
:100B34004F4B9000057406122C857406020E311278
:100B44002C78F97411122C72F990000112179D522D
:100B54005F4F4B900005740C122C857412020E31F9
:100B6400122D12C2B6122D5AFF240DF582E43EF561
:100B740083E0543FF5B0EF122BDCF990000112171B
:100B84009D575F4F4B9000057406122C8574060226
:100B94000E31122D12122C75122CED902416F01217
:100BA4002C70F990000112179D575F4F4B122C8047
:100BB400120E84120EAE020D33122D12122C751267
:100BC4002D7690241B122D3E90241C122D7D9024F2
:100BD4001D122D0B90241EF0122C70F9900001129E
:100BE400179D575F4F4B122C80120E847B017A2481
:100BF400791B124979020D33122D12122C75122D04
:100C040076902417122D3E902418122D7D902419CD
:100C1400122D0B90241AF0122C70F9900001121767
:100C24009D575F4F4B122C80120E937B017A2479CF
:100C34001712499C020D33122D12122C75122CED31
:100C4400902416F090000912150F902417F09000CC
:100C54000A12150F902418F090000B12150F90240F
:100C640019F090000C12150F90241AF090000D1238
:100C7400150F90241BF090000E12150F90241CF0F9
:100C840090000F12150F90241DF090001012150FF4
:100C940090241EF0122C70F990000112179D575FDA
:100CA4004F4B122C80120E93122C75122D537B571E
:100CB4007A4E79687843C31216EC7013120EAE7A2A
:100CC40024791712499C7A24791B12497980069059
:100CD40024A57464F07B01020D33122D12122C75BD
:100CE400122D7690240D122D3E90240E122D7D90FF
:100CF400240F122D0B902410F090000912150F9060
:100D04002411F090000A12150F902412F0122C7086
:100D1400F990000112179D575F4F4B122C807406F7
:100D2400F0120EA27B017A24790D1245E57B017A3B
:060D3400247907024A04C5
:100D3A00E4902437F0A3F090011504F0122C75F911
:100D4A001214F6C394064015122D3F7004FEFF805C
:100D5A00047E007F01902437EEF0A3EFF090243751
:100D6A00A3E02424122C72F990000112179D525FFD
:100D7A004F4B122D6E90242EE0FEA3E0FFC3942069
:100D8A00EE9400503F7B0174072FF974243EFA1247
:100D9A0014F6FF122C752405F9E43AFA902437E088
:100DAA00FCA3E0FD90242EE0F8A3E02DFDE83CFC36
:100DBA00E92DF9EA3CFAEF12153C122D8470B612AD
:100DCA002D8B80B1D3902438E09400902437E0949E
:100DDA0000400C122C75F9900005742012154E1261
:100DEA002D1BC003C002C001122C75F91214F6247F
:100DFA0001FEE43390243DF0A3CEF0902427E0FFD7
:090E0A00D001D002D003020E5108
:100E1300122D1222122D12122C65F99000011217B5
:100E23009D575F4F4B900005E4122C857406F080AC
:100E33001D122D12122C75F97404122C72F99000E4
:100E43000112179D5F457272122C887405F0120E01
:100E5300A222902427E0FF024AEF902427E0FF120A
:100E63004A41902427E0FFA3E0FAA3E0FB90243D4E
:100E73007420F07D01023CDB902427E0FF1247FF42
:100E8300227406F012338990242CEEF0A3EFF022A3
:100E93007406F012338990242CEEF0A3EFF02212A3
:100EA300338990242CEEF0A3EFF0227B017A24798E
:050EB300131249BF22EB
:1040C600446973636F76657279554450203A20527D
:1040D6006563656976656420256420627974657315
:1040E6002066726F6D202562752E2562752E2562FB
:1040F600752E256275203D00202530326258000D50
:104106000A00446973636F76657279554450203AA4
:1041160020446973636F766572792042726F6164B9
:10412600636173742044657465637465640D0A0085
:10413600446973636F76657279554450203A2073EB
:084146006F636B65740D0A0044
:104A7800EEF0A3EFF0A3EBF0A37424F0A37429F0F5
:0A4A8800A322F582E43CF583E0224E
:08371400902427EEF0A3EFF072
:10371C007F037E471249EFEF700302381824DE60F6
:10372C00030238287F07124425D3EF9400EE94004F
:10373C005003023828902427E0FCA3E0AA04F97B6C
:10374C0001C00390243A124A78EBF0A37424F0A33E
:0A375C00742DF0D0037F071230C572
:10376600E490242FF090242FE0C39FE49E5005E0C0
:0437760004F080F1EA
:10377A00EF64084E6003023828902427E0FCA3E097
:10378A00FDF5828C83E064B26003023828A3E0640A
:10379A00D46003023828902427A3E0F5828C83A3FF
:1037AA00A3E064E570788D828C83A3A3A3E0640C04
:1037BA00706C902427A3E02404124A8A6426705E5F
:1037CA00ED2405124A8A64D47054902427A3E02475
:1037DA0006124A8A64777046ED2407124A8A6446BA
:1037EA00703C902427A3E0AA04F97B01C00390242B
:1037FA0038124A7874CAF0A374DEF0D0037F071235
:10380A002D927B017A2479171248E40248BAE4908F
:0E381A00243DF07BDF7ACA7D027F07123CDB83
:01382800227D
:1035F3000D0A4143434553204554482D44494F2D1B
:1036030034382055706C6F616420506F727420439E
:103613006F6E6E65637465640D0A0055706C6F613F
:103623006420446174616772616D3A2025730D0AE9
:10363300005374617475733D382C206C696E656C2E
:10364300656E6774683D25303262782066756C6CF0
:10365300646174616772616D3D2530326278206305
:103663006F6D706172653D2530326278005374610D
:103673007475733D31302C206C696E656373756DA1
:103683003D2530326278206373756D5F63616C63CF
:103693003D25303262782C2073756D3D25303262C2
:1036A30078200D0A006C61756E6368696E67206629
:1036B3006C61736820636F7079206F7065726174D9
:1036C300696F6E2066726F6D20253034780D0A00A5
:1036D3000D0A666C61736820636F7079207265747C
:1036E30075726E65643F213F21213F20756E6578B9
:1036F3007065637465642073686F756C64206861BA
:10370300766520637261736865642E2E2E2E0D0A12
:0137130000B5
:0C45CB0041245F00412460004124610095
:103F1500F0902433E0FBA3E0FAA3E022902427E00D
:103F2500FF90242AE0FCA3E0AA04F97B0122FAA968
:103F35000790243A7401F0A3EAF0A3E9F022902453
:103F450068E090242EFFE0FCA3E0FDC39FEC221265
:103F550014F6FFFD3395E0FC90247EE02DF09024CF
:103F65007DE03CF022E02430F090247DE034002216
:103F7500A3E0FDA3E090243DCD222DFD90242AE071
:103F85003400FAA9057B0122FE12150F7C002400DE
:103F9500FFEC3E221214F6FFC3648094C122D39431
:0C3FA50000EE9400229001157401F0223F
:10450D00E4FE123F5412490A5011123F995006EF22
:10451D0024D0FE80061214F624C9FE740129F9E494
:10452D003AFA123F54EEC454F0FE12490A501312D7
:10453D003F995007EF24D02EFE80071214F624C9A0
:0A454D002EFE902481E02EF0AF0650
:014557002241
:10476D00902437EB123F3B902437123F192402F966
:10477D00E43AFA12450D7E00C006C00790243712A8
:10478D003F19F912450DEFFCD0E02400FFD0E03CBD
:02479D00FE22FA
:100EB800902427EFF0A3ECF0A3EDF0A3EAF0A3EB66
:010EC800F039
:100EC900F9902430123F39A3123F39E4A3F090245A
:100ED90027E0FF124B1AEF700302139E24ED7003F3
:100EE9000213BC24F770030213782405600302136C
:100EF900C4902427E0FF124B90EF30E0189024278C
:100F0900E0FF7D01124B79E490245FF07BFF7A3595
:100F190079F312193E1213C5123FA35003020FB9F8
:100F290090245FE0702F123F2190243DE4F0A30448
:100F3900F0123DAA90242CEEF0A3EFF090242AE0C1
:100F4900FEA3E0F5828E83E0902460F090245F7424
:100F590001F0020FB9902460E0FFD390242DE09FA7
:100F690090242CE09400902427E0FF90245FE0FD7A
:100F790090242BE0500B123F7F90242C123F768057
:100F89000C123F7F902460E0FD90243DE41213D6BB
:100F990090242CA3E0FF90245FE02FF0A3E0C39FEF
:100FA900F0700D90245FE0902436F0E490245FF017
:100FB900902436E07003021372902430123F19F91D
:100FC9009000011217101217C1106B554461741269
:100FD900C55546696E0FE855706C640000137212AE
:100FE9003FAAE4902460F0A3F09024A4F090248117
:100FF900F090247DF0A3F0902466F0A3F090247B78
:10100900F0A3F0902464F0A3F074FF902462F0A39D
:10101900F09024617401F09024A4F0900006121558
:101029000F900005123F8D902466F0A3EFF0900019
:101039000812150FFE90000712150F2400FFEC3E51
:101049004F60069024A47420F0902430123F19F9BF
:1010590090000A12150F900009123F8D90247F020B
:10106900136E123FAA902461E064016003021372B7
:101079009024A4E0FF640160030212BD123F16F937
:1010890090000512150F643A6008EF44029024A4F9
:10109900F02290247EE0243A123F6DF090000C1269
:1010A90015C764307004E5F0643060089024A4E04A
:1010B9004404F02290247E123F6AF0A3123F6A1280
:1010C9003F152406F9E43AFA12450D902468EF1207
:1010D9003F152408F9E43AFA12476D902479EEF0A5
:1010E900A3EFF0902468E0F92FFFE43ECF24FFCF6F
:1010F90034FFFEC3902465E09F902464E09E500570
:10110900EEF0A3EFF0902462E0FEA3E090247912C0
:101119003F4A9E5008902462ECF0A3EDF0902436EB
:10112900E0FD24F0FBE434FFFAE975F002A46B70EA
:1011390003E5F06A603F9024A4E04408F090242A73
:10114900E0FEA3E0FF2DF582E43EF583E4F0EF2411
:1011590005FFE43E123F331213F47A3679349024B2
:1011690068E025E090243AF0902436E090243BF0A2
:1011790024F002122DE490242EF0A3F0123F4394A0
:1011890000503B123F16240EF9E43AFAED25E0FF30
:10119900EC33FEE92FF9EA3EFA12450D90242EE0D0
:1011A900FCA3E02469F58274243CF583EFF09024D4
:1011B9002FE004F070C690242EE004F080BE123FA8
:1011C90016240EF9E43AFA902468E075F002A4298D
:1011D900F9EA35F0FA12450D902482EFF090248156
:1011E900E060469024A4E04410F0902436E0FF909B
:1011F900242AE0FCA3E0FD2FF582E43CF583E4F02A
:10120900ED2405FFE43C123F331213F47A3679706A
:10121900902482E0FF90243AF0902481E0FE90240B
:101229003BF0EF2EA3F002193E90247CE004F0700D
:101239000690247BE004F0902466E0FEA3E0FF9092
:10124900247BE0B5062AA3E0B507259024A4E05441
:10125900FEF090247DE0FEA3E0FF902480E02FFFC4
:1012690090247FE03E4F60089024A4E04440F0229F
:10127900E490242EF0A3F0123F439400400302139C
:101289007274692DF58274243CF583E0FF90247A09
:10129900E02DFD902479E03CFCE42DF58274803C3E
:1012A900F583EFF090242FE004F070CB90242EE02A
:1012B90004F080C39024A4E04480F022123FAAE401
:1012C900902461F09024A4E09024307049123F19D1
:1012D900F9740412153C902430123F19F990000159
:1012E90012179D575F4F4B123F2190243DE4F07434
:1012F900051213E6C2AF7BFF7A3679A890243A74B7
:1013090070F0A3E4F012193E1270007BFF7A36796F
:10131900D312193E8031123F19F9740512153C9008
:101329002430123F19F990000112179D5F4572721E
:101339009024A4E090000512154E123F2190243DFF
:10134900E4F074061213E6E490245FF01213C51258
:101359003FA34015123F21123F75F0A3EDF0123D56
:10136900AA90242CEEF0A3EFF0E4902436F022901A
:101379002427E0FF12442590242CEEF0A3EFF0126D
:101389003FA34009123F21123F751213D69024271B
:10139900E0FF024AEF902427E0FF124A41902427F8
:1013A900E0FFA3E0FAA3E0FB90243D7420F07D0167
:0B13B900023CDB902427E0FF1247FFFE
:1013C40022902427E0FF12442590242CEEF0A3EF72
:1013D400F022F0A3EDF0123DAA90242CEEF0A3EF3E
:1013E400F022A3F012338990242CEEF0A3EFF02224
:0C13F4007BFF7A36791E12193E7BFF2227
:1042A30054696D65206F75742E0D0A007374617403
:1042B300655F646863705F726571756573742025EB
:1042C30064007374617465203A2053544154455F0C
:1042D300444843505F444953434F5645520D0A00E7
:1042E3004448435020446576696365204E616D659B
:1042F3003A20000D0A004661696C3A53616D6549C5
:04430300500D0A004F
:0D45D70041213900412370004221370000CE
:1023FC00F0902432E475F001121586FE743825F045
:10240C00F58274223EF5837401F0902432E475F069
:10241C0001121586FE743825F0F58274223EF58380
:10242C007403F0902432E475F001121586FE7438B2
:10243C0025F0F582742222E0FF902432E475F0013D
:10244C00021586E4F0A3F090214C04F0A3F0A374E1
:10245C0006F0E4A3F0902148E0FCA3E0FDA3E0FE2D
:10246C00A3E0FF902150121760E4902154F0A3F0E8
:10247C00A37480F0A3E4F0FE7F04FD7B017A217944
:10248C00581217FB7E007F047D007B017A21795C5A
:10249C001217FB7E007F047D007B017A217960128C
:1024AC0017FB7F047A2179647E007D007B01021783
:1024BC00FB902375E0FCA3E0FDA3E0FEA3E0240564
:1024CC0090213BFFE43EFEE43DFDE43CFC02176042
:1024DC0085F082F583E0902431F0A3E0FEA3E022A6
:1024EC007E007F407D007B017A2179781217FB7F7B
:1024FC00807A2179B87E007D007B010217FB902148
:10250C0048E0FCA3E0FDA3E0FEA3E02401FFE43ED1
:10251C00FEE43DFDE43CFC9021481217607D01E493
:10252C0022902375E0FCA3E0FDA3E0FEA3E022745F
:10253C00102EF582E43424F583E022902428E0FF69
:10254C002413F582E43424F58322A3F0902379E05C
:10255C00FDA3E090243DCDF0A3EDF07B017A217931
:10256C004C2290242CE0FEA3E0FF223EF583EDF0FC
:10257C0090242DE004F022F583EEF0902428E00462
:10258C00F0E022E490243DF07B44FA7D02FF22E04F
:10259C00FF9024387402F0A37428F0A37401F0A304
:1025AC0022F58274243EF583E0FD74682FF5827465
:1025BC0021223EF5837401F02290242CE004F022B9
:1025CC00540F75F00A84E5F02274382FF5827422CA
:1025DC003EF583E422E490242CF0A3F022E0F8A34F
:1025EC00E0F9A3E0FAA3E0FB2274292FF582742111
:1025FC003EF58322E4902139F090212404F0223E10
:10260C00F5837463F090242F22902379E4F0A37463
:03261C0043F02266
:034BB800B2B7226F
:0528360090242AEFF0E0
:10283B0090242F12244F7F107A2179681224B4E44C
:10284B00FFFE740D2F1225AD3EF583EDF00FBF008B
:10285B00010EEF64064E70EA1224EC90242F122422
:10286B003212260B1224323EF5837482F090242F01
:10287B001224323EF5837453F090242F122432121B
:10288B00260B1224323EF5837435F090242F12243C
:10289B00321225BE90242F1224321225BE90242FE3
:1028AB001224323EF583743DF090242F1224323ED5
:1028BB00F5837407F090242F1224321225BE902436
:1028CB000DE0FF90242F122448FC12243A3CF58390
:1028DB00EFF090240EE0FF90242F122448FC1224DA
:1028EB003A3CF583EFF090240FE0FF90242F122455
:1028FB0048FC12243A3CF583EFF0902410E0FF9053
:10290B00242F122448FC12243A3CF583EFF0902438
:10291B0011E0FF90242F122448FC12243A3CF5833B
:10292B00EFF0902412E0FF90242F122448FC122485
:10293B003A3CF583EFF090242F1224323EF583744A
:10294B000CF090242F1224323EF583740EF0E4FE2B
:10295B00FF1225F5E0FD90242F122448FA12243A99
:10296B003AF583EDF00FBF00010EEF640E4E70E1F0
:10297B0090242F1224323EF5837437F090242F12BB
:10298B0024323EF5837405F090242F122432122545
:10299B00BE90242F1224323EF5837403F090242F23
:1029AB001224323EF5837406F090242F1224323E0B
:1029BB00F583743AF090242F1224323EF583743B46
:1029CB00F090242F1224323EF58374FFF090242FC5
:1029DB00E0FEA3E0FFC3EF9438EE9401500B1225F9
:1029EB00D5F00FBF00010E80EC122615E4FF7E041C
:1029FB0090242B74FFF0A3DEFC90242A12259B74E9
:0A2A0B0024F0742B122556022D92C0
:081C380090242AEFF0A3EDF067
:101C400090243212244F7F107A21796812250112D4
:101C500025E112256E240D1225AD12257770031291
:101C600025C590242CE07004A3E0640670E41224DF
:101C7000EC12242F3EF583746312242E3EF58374F8
:101C80008212242E3EF583745312242E3EF5837463
:101C90006312242E3EF58374351223FC3EF58374C3
:101CA0003D12242E3EF583740712242E1225BE9079
:101CB000240D122443FC12243A3CF583EFF09024C7
:101CC0000E122443FC12243A3CF583EFF090240FCB
:101CD000122443FC12243A3CF583EFF090241012B6
:101CE0002443FC12243A3CF583EFF0902411122493
:101CF00043FC12243A3CF583EFF090241212244363
:101D0000FC12243A3CF583EF12242E3EF583743204
:101D100012242E3EF5837404F090242BE0FF6038EB
:101D2000902140E0FE122445FC12243A3CF583EE5B
:101D3000F0902141E0FE122445FC12243A3CF58348
:101D4000EEF0902142E0FE122445FC12243A3CF5CC
:101D500083EEF09021438036902413E0FE12244558
:101D6000FC12243A3CF583EEF0902414E0FE122499
:101D700045FC12243A3CF583EEF0902415E0FE1267
:101D80002445FC12243A3CF583EEF0902416E0FE44
:101D9000122445FC12243A3CF583EEF0122445FC53
:101DA00012243A3CF5837436F0122445FC12243A8E
:101DB0003CF5837404F0EF6032902118122443FC48
:101DC00012243A3CF583EFF0902119122443FC12BF
:101DD000243A3CF583EFF090211A122443FC12249C
:101DE0003A3CF583EFF090211B8030902371122450
:101DF00043FC12243A3CF583EFF090237212244303
:101E0000FC12243A3CF583EFF0902373122443FC38
:101E100012243A3CF583EFF0902374122443FC1211
:101E2000243A3CF583EFF012242F3EF583740C1214
:101E3000242E3EF583740EF01225E112256EC39414
:101E40000EEE940050181225F5122443FC12243A89
:101E50003CF583EF12257B70E21225C580DD12244C
:101E60002F3EF583743712242E3EF583740512231A
:101E7000FC3EF583740612242E3EF583743A122438
:101E80002E3EF583743B12242E3EF58374FFF090B2
:101E90002432E0FFA3E090242CCFF0A3EFF0122532
:101EA0006EC39438EE9401500D1225D512257B7027
:101EB000ED1225C580E812261590242BE06030E451
:101EC000A3F0A3F012256E2418F58274213EF58349
:101ED000E0FD742E2FF582742412257770031225ED
:101EE000C590242CE07004A3E0640470D780241211
:101EF00025E112256EC39404EE94005016742E2F23
:101F0000F58274243EF58374FF12257B70E412255C
:101F1000C580DF90242A12259B7424F0742E12258C
:041F200056022D92A6
:102A1500E4FB90243AECF0A3EDF00BA3EBF0A374E8
:102A250024F0A3742AF0A3EBF0A37424F0A3742E6E
:102A3500F07A21794C1230C5AA06AB0790242EE016
:102A45007004A3E06443705DFF740D2FF582E434D8
:102A550024F583E0FE74682FF582E43421F583E0E4
:102A65006E60037F00220FEFB406DEE4FF74602F73
:102A7500F582E43421F583E0FE74712FF582E434A8
:102A850023F583EEF00FEFB404E3E4FF745C2FF558
:102A950082E43421F583E0FE74132F12254EEEF007
:102AA5000FEFB404E7E4902430F09024327421F061
:102AB500A3744CF0E024F0F0902432E03400F0EB05
:102AC5002410FFEA34FFFEA3E02FFF902432E03EFE
:102AD500902434F0A3EFF0902434E0FEA3E0FFC38C
:102AE500902433E09F902432E09E4003022BD612BF
:102AF500244885F082F583E07003022BC11460320F
:102B050024FE604324FD605324D3606324FE600DDE
:102B150014607C24376003022BB1022BD69024323B
:102B25001224481224DCF5828E83E0902430F002D2
:102B35002BC19024321224481224DCAA06F97B0109
:102B450078177C24022BA69024321224481224DC08
:102B5500AA06F97B01781B7C248046902432122436
:102B6500481224DCAA06F97B0178447C2180329046
:102B750024321224481224DCF5828E83E0FCA3E083
:102B8500FDA3E0FEA3E0FF90211C121760802D90AD
:102B950024321224481224DCAA06F97B0178717CC0
:102BA500237D017E007F041214D080109024321200
:102BB500244885F082F583E0902431F0902431E0BB
:102BC500FF902433E02FF0902432E03400F0022A05
:062BD500DC902430E0FF5B
:012BDB0022D7
:10403D00902139E0C3940A505412252DFF90213B55
:10404D00E0F8A3E0F9A3E0FAA3E0FBC31216EC50ED
:10405D006790237512176C000000001224BD90218B
:10406D0039E004F0902124E024FE600D24FE600D63
:10407D0024037044E4FF022836E4FD800C12258FE2
:10408D00123CDBBF01F712250AFF021C387BFF7AB9
:10409D004279A312193E9023707401F0902375128A
:1040AD00176C000000001224BDE4902139F0FF12BE
:0940BD0028369021247401F02240
:103C01007D80E4FFFE124B0590241BE0FD7F011235
:103C11004B0590241CE0FD7F02124B0590241DE012
:103C2100FD7F03124B0590241EE0FD7F04124B051E
:103C3100902417E0FD7F05124B05902418E0FD7FCD
:103C410006124B05902419E0FD7F07124B059024C5
:103C51001AE0FD7F08124B05902413E0FD7F0F123F
:103C61004B05902414E0FD7F10124B05902415E0C4
:103C7100FD7F11124B05902416E0FD7F12124B05BA
:103C810090240DE0FD7F09124B0590240EE0FD7F8D
:103C91000A124B0590240FE0FD7F0B124B05902477
:103CA10010E0FD7F0C124B05902411E0FD7F0D12F9
:103CB1004B05902412E0FD7F0E124B057D037F1909
:103CC100124B0590242F7401F0A37401F0A3740327
:0A3CD100F07B017A01790B02261F37
:1021C300E4FFFE124425D3EF9400EE9400400EADDD
:1021D30007AC06E4FF122A15902429EFF09021247E
:1021E300E024FE605D1470030222FC1470030223DA
:1021F30081240360030223FB902429E06402703FDF
:10220300FDFF121C389021247402F07BFF7A42797F
:10221300AFE0FF90243AE4F0A3EFF012193E9023CD
:1022230074E0902123F0902373E0902122F0902317
:1022330072E0902121F0902371E0902120F022029E
:1022430023F8902429E064057057123C01E490249C
:1022530028F0902428E0FF2471F582E43423F583E9
:10226300E0FE74182FF582E43421122583B404E2CE
:10227300E4902428F0122547E0FE74402FF582E411
:102283003421122583B404ED9021247403F09023A8
:102293007512176C000000001224BDE4902139F080
:1022A30022902429E06406704D902374E0FF90216E
:1022B30023E06F60030223FB902373E0FF9021224E
:1022C300E06F60030223FB902372E0FF902121E083
:1022D3006F60030223FB902371E0FF902120E06FE6
:1022E30060030223FB90237512176C000000001299
:1022F30024BD122600220223F874FFFFFEFDFC908A
:10230300211C1225E9C31216EC70030223FBE47BA4
:1023130002FAF9F890211C122530FF12165A902365
:10232300751225E9D31216EC50030223FBE4902423
:1023330029F0902428F0122547E0FE74252FF5821A
:10234300E43421122583B404ED12258F123CDBBF44
:1023530001F712250AFF121C389021247404F0900F
:10236300237512176C0000000012252D2405FFE4CD
:102373003EFEE43DFDE43CFC90213B0217609024CB
:1023830029E06405704F902139F0FF902428F090E4
:102393002428E0FE12254CE0FD74252EF582E4345A
:1023A30021F583E06D60047F018006122587B40464
:1023B300DEEF600D90237512176C00000000123CD5
:1023C3000190237512176C000000001224BD9021A8
:1023D300247403F022902429E0B406199023751283
:1023E300176C000000001224BD1226007BFF7A4206
:0823F30079C502193E12403DBC
:0123FB0022BF
:103E6D009021297445F0A37454F0A37448F0A37401
:103E7D0044F0A37449F0A3744FF0A37434F0A37409
:103E8D0038F0E4FE12253BC4540FFFC3940A4008DA
:103E9D00EF1225CE2441800912253BC41225CC24D6
:103EAD0030FFEE25E02431F582E43421F583EFF087
:103EBD0012253B540FFFC3940A4008EF1225CE2460
:103ECD0041800812253B1225CC2430FFEE25E0243D
:103EDD0032F582E43421F583EFF00EEE640370A425
:103EED007BFF7A4279E312193EE4FE74292EF582A6
:103EFD00E43421F583E0FF124B990EEEB40EEC7B0A
:083F0D00FF7A4279F602193E29
:10436900123E6D90214812176C1234566512258F32
:10437900123CDBBF01F7E4FF1228369021247401B7
:10438900F0E490213AF090237512176C00000000B8
:104399001224BDE4902139F090011304F0902124F6
:1043A900E0640360191221C390213AE0C3940240EA
:1043B900037F0022902370E0B401E27F00227F0195
:0143C90022D1
:104A9200C2AFC28CC28D758901758A5B758CE3C207
:084AA200B9D2A9D2AFD28C22D7
:03000B0002423B73
:10423B00C0E0C0F0C083C082C0D075D000C000C049
:10424B0004C005C006C007C28CC28D745B258AF5FD
:10425B008A74E3258CF58CD28C900113E0B4012386
:10426B00902137122448FEC3E5F09488EE94134056
:10427B0012902137E4F0A3F012252D240190237521
:10428B001224CFD007D006D005D004D000D0D0D088
:08429B0082D083D0F0D0E032A4
:03000000023FB10B
:0C3FB100787FE4F6D8FD758121023FF80E
:10140000E709F608DFFA8046E709F208DFFA803ECE
:1014100088828C83E709F0A3DFFA8032E309F608BB
:10142000DFFA8078E309F208DFFA807088828C8323
:10143000E309F0A3DFFA806489828A83E0A3F608D7
:10144000DFFA805889828A83E0A3F208DFFA804CB1
:1014500080D280FA80C680D4806980F28033801088
:1014600080A680EA809A80A880DA80E280CA8033F1
:1014700089828A83ECFAE493A3C8C582C8CCC58369
:10148000CCF0A3C8C582C8CCC583CCDFE9DEE78039
:101490000D89828A83E493A3F608DFF9ECFAA9F0B8
:1014A000EDFB2289828A83ECFAE0A3C8C582C8CC0E
:1014B000C583CCF0A3C8C582C8CCC583CCDFEADE27
:1014C000E880DB89828A83E493A3F208DFF980CC89
:1014D00088F0EF60010E4E60C388F0ED2402B40482
:1014E0000050B9F582EB2402B4040050AF23234529
:0614F000822390145073EA
:1014F600BB010689828A83E0225002E722BBFE02F4
:09150600E32289828A83E4932226
:10150F00BB010CE58229F582E5833AF583E0225091
:10151F0006E92582F8E622BBFE06E92582F8E222DB
:0D152F00E58229F582E5833AF583E49322F5
:10153C00BB010689828A83F0225002F722BBFE018E
:02154C00F32288
:10154E00F8BB010DE58229F582E5833AF583E8F0D3
:10155E00225006E92582C8F622BBFE05E92582C87F
:02156E00F22267
:10157000C5F0F8A3E028F0C5F0F8E5821582700206
:061580001583E038F022A3
:10158600A3F8E0C5F025F0F0E58215827002158318
:06159600E0C838F0E82275
:10159C00BB010A89828A83E0F5F0A3E0225006871A
:1015AC00F009E71922BBFE07E3F5F009E3192289DC
:0B15BC00828A83E493F5F0740193220F
:1015C700BB0110E58229F582E5833AF583E0F5F062
:1015D700A3E0225009E92582F886F008E622BBFE3F
:1015E7000AE92582F8E2F5F008E222E5832AF58385
:0815F700E993F5F0A3E993224A
:1015FF00BB010A89828A83F0E5F0A3F0225006F737
:0F160F0009A7F01922BBFE06F3E5F009F3192233
:10161E0075F008758200EF2FFFEE33FECD33CDCC83
:10162E0033CCC58233C5829BED9AEC99E582984006
:10163E000CF582EE9BFEED9AFDEC99FC0FD5F0D6E3
:10164E00E4CEFBE4CDFAE4CCF9A88222B800C1B90D
:10165E000059BA002DEC8BF084CFCECDFCE5F0CB4B
:10166E00F97818EF2FFFEE33FEED33FDEC33FCEB84
:10167E0033FB10D703994004EB99FB0FD8E5E4F93F
:10168E00FA227818EF2FFFEE33FEED33FDEC33FC2C
:10169E00C933C910D7059BE99A4007EC9BFCE99A20
:1016AE00F90FD8E0E4C9FAE4CCFB2275F010EF2F65
:1016BE00FFEE33FEED33FDCC33CCC833C810D70765
:1016CE009BEC9AE899400AED9BFDEC9AFCE899F8A0
:0E16DE000FD5F0DAE4CDFBE4CCFAE4C8F92233
:1016EC00EB9FF5F0EA9E42F0E99D42F0E89C45F054
:0116FC0022CB
:1016FD00E8600FECC313FCED13FDEE13FEEF13FFCB
:03170D00D8F122EE
:10171000BB010DE58229F582E5833AF58302183392
:101720005007E92582F8021827BBFE07E92582F851
:1017300002183FE58229F582E5833AF58302184BCA
:101740007401FF3395E0FEFDFC080808E6CF2FF694
:1017500018E6CE3EF618E6CD3DF618E6CC3CF6226D
:0C176000ECF0A3EDF0A3EEF0A3EFF022FC
:10176C00A8828583F0D083D082121783121783123C
:10177C001783121783E473E493A3C583C5F0C58361
:10178C00C8C582C8F0A3C583C5F0C583C8C582C8C7
:01179C00222A
:10179D00BB010DE58229F582E5833AF58302176CCD
:1017AD005007E92582F802185BBBFE07E92582F890
:0417BD000218742278
:1017C100D083D082E4937012740193700DA3A3931C
:1017D100F8740193F5828883E4737402936C701238
:1017E1007403936D700C7404936E70067405936F9B
:0A17F10060DDA3A3A3A3A3A380CA95
:1018D300E508243AF582E43424F583E005082290F0
:1018E300243730070390243AE475F00112188D026F
:1018F30014F62000E97F2ED2008018EF540F2490B5
:10190300D43440D4FF30040BEF24BFB41A00500387
:101913002461FFE50960021509050CE50C70020559
:101923000B30070E902437E475F00112188DEF0287
:10193300153C024B997403D2078003E4C207F508F0
:101943009024371218A4E4F509F50BF50CE50960AA
:10195300077F2012191680F5750AFFC201C200C263
:1019630002C203C205C206C2081218E2FF700D309C
:1019730007057F00121927AF0CAE0B22B4255FC2F7
:10198300D5C2041218E2FF24D0B40A00501A75F02D
:101993000A780930D50508B6FF0106C6A426F62045
:1019A300D5047002D20380D924CFB41A00EF5004B7
:1019B300C2E5D204021B28D20180C6D20080C0D265
:1019C3000280BCD2D580BAD20580B47F201219160A
:1019D3002002077401B5090040F11218D3FF121950
:1019E30016021950D208D20680951218D3FB12188A
:1019F300D3FA1218D3F94A4B700679F97A1B7BFF95
:101A030020022EE509602A7E008E8275830012155E
:101A13000F60060EEE650A70F0C2D5EBC0E0EAC0B7
:101A2300E0E9C0E0EE121B6FD0E0F9D0E0FAD0E0BD
:101A3300FB1214F6FF60AAEBC0E0EAC0E0E9C0E0E5
:101A4300121916D0E02401F9D0E03400FAD0E0FBFB
:101A5300E50A0460DCD50AD980877BFF7A1B796BA2
:101A6300D202809C791080027908C206C2088008DD
:101A7300D2D5790A8004790AC2D5E50A047002F541
:101A83000AE4FAFDFEFF1218D3FC7B0820011312AF
:101A930018D3FD7B1030000A1218D3FE1218D3FF9F
:101AA3007B20EC3382D592D55013C3E43000069FDC
:101AB300FFE49EFEE42001039DFDE49CFCE4CBF8DF
:101AC300C201EC700CCFCECDCCE824F8F870F380D3
:101AD30017C3EF33FFEE33FEED33FDEC33FCEB3393
:101AE300FB994002FB0FD8E9EB300105F8D0E0C4C5
:101AF30048B201C0E00AEC4D4E4F78207B0070C223
:101B0300EAB50A0040BCC0E0121B71D0F0D0E0205F
:101B13000104C4C0E0C4B201C0F01218FFD0F0D574
:101B2300F0EB0219501218AD19ED531A675819BE8C
:101B33004C19BA421A6B4F1A73441A734919D34397
:081B43001A79551A5D461A5D7E
:101B4B00451A5D471C195019C22D19C62E19E92BC0
:101B5B0019CA2319E7201C022A198248000019E12F
:101B6B003F3F3F00790AA2D5200314300509B91075
:101B7B00020404B9080104A2D52006025001042076
:101B8B0002689202B509005034C0E07F203003197F
:101B9B007F30A20272067205500F121BC8C202C21E
:101BAB0006C205C2087F30800F300503E9C0E01282
:101BBB001916300503D0E0F9D0E0B509CC30051784
:101BCB007F30B9100C1219167F583004077F7880BC
:101BDB0003B908031219163002057F2D0219167F5F
:101BEB00202008F87F2B2006F322920280CF286E4C
:101BFB00756C6C2900D2011218D33001F8C2017830
:101C0B000930D50108F60219822D50434958121894
:101C1B00D32403B405004001E4901C14931219075C
:0D1C2B00743A121907D203750904021A67F2
:10490A00EFC394414005EF94474016EFC3946140CA
:10491A0005EF9467400BEFC394304008EF943A5088
:06492A0003D38001C3224B
:1017FB00EF4E6012EF60010EEDBB010B89828A8305
:10180B00F0A3DFFCDEFA2289F05007F709DFFCA911
:0C181B00F022BBFEFCF309DFFCA9F02268
:103FBD00021F24E493A3F8E493A34003F68001F2D7
:103FCD0008DFF48029E493A3F85407240CC8C33305
:103FDD00C4540F4420C8834004F456800146F6DFD4
:103FED00E4800B01020408102040809045A1E47E7E
:103FFD00019360BCA3FF543F30E509541FFEE493C9
:10400D00A360010ECF54C025E060A840B8E493A38F
:10401D00FAE493A3F8E493A3C8C582C8CAC583CABA
:10402D00F0A3C8C582C8CAC583CADFE9DEE780BE72
:0145E40000D6
:0C182700E6FC08E6FD08E6FE08E6FF22ED
:0C183300E0FCA3E0FDA3E0FEA3E0FF2228
:0C183F00E2FC08E2FD08E2FE08E2FF22E5
:10184B00E493FC740193FD740293FE740393FF22E3
:10185B00D083D082E493F608740193F60874029354
:09186B00F608740393F67404738B
:10187400D083D082E493F208740193F20874029343
:09188400F208740393F27404737A
:10188D00F8E0FBA3A3E0F925F0F0E58215827002E4
:07189D001583E0FA38F02288
:0918A400EBF0A3EAF0A3E9F02245
:1018AD00D083D082F8E4937012740193700DA3A3CA
:1018BD0093F8740193F5828883E4737402936860DE
:0618CD00EFA3A3A380DFDE
:00000001FF
